:020000040000FA
:10000000000003018B001B280B1C0900861006153D
:100010000608F039A3000310A30CA30C23082A023E
:10002000031916282308AA005021742106080B1072
:10003000061186140900850107309F008316E03001
:100040008500F130860081018312083005168B008F
:10005000061C52281830850006118610C830A200F0
:10006000061567216721A20B30288511A8012810E9
:1000700067216721672167210608F039AA0003106C
:10008000AA0CAA0C502174216721672174216721D1
:1000900006118B1700008614630000000000861014
:1000A00000004A288614113000233F3000238610B8
:1000B000B42152302B020319BD2872302B020319D0
:1000C000BD2847302B0203192A2867302B02031959
:1000D00095287E300023B421DD21AA000F30AA0527
:1000E00098300023A401A501A601A7019B21E530BA
:1000F00000230A3003142A02031C81282A08373EF1
:1001000083282A08303EFF212030FF212030FF21A4
:100110001722BD300023B42157302B020319982831
:1001200077302B02031998285528D33000232A282A
:10013000AA0DAA0D3C30AA052A08033EB5202408C2
:10014000B92050222A08023EB5202508B9205022A5
:100150002A08013EB5202608B92050222A08003E70
:10016000B5202708B9205022552883169B008312FA
:10017000080083169A008312080061226122303041
:10018000FF212030FF210030AA00502117226122D8
:100190003130FF212030FF210430AA0050211722E6
:1001A00061223230FF212030FF210830AA00502187
:1001B000172261223330FF212030FF210C30AA00AA
:1001C0005021172261223430FF212030FF211030CE
:1001D000AA005021172261223530FF212030FF2153
:1001E0001430AA005021172261223630FF2120301E
:1001F000FF211830AA005021172261223730FF2139
:100200002030FF211C30AA005021172261223830F3
:10021000FF212030FF212030AA0050211722612227
:100220003930FF212030FF212430AA00502117222D
:1002300061224130FF212030FF212830AA005021C7
:10024000172261224230FF212030FF212C30AA00EA
:100250005021172261224330FF212030FF2130300E
:10026000AA005021172261224430FF212030FF21B3
:100270003430AA005021172261224530FF2120305E
:10028000FF213830AA005021172261224630FF2179
:100290002030FF213C30AA0050211722612255282E
:1002A00003302A076121A40002302A076121A5003A
:1002B00001302A076121A60000302A076121A7002A
:1002C000080083169B001C141A08831208000615E8
:1002D0009D30A100000000000000000000000000B0
:1002E000A10B6A290611080061221722240889211E
:1002F000250889212608892127088921280889219C
:100300000511851400000000000085100510000094
:100310000800A3000830A00000000511A30C031C76
:10032000051003180514000000000515000000006A
:10033000A00B8C290800B4212B080D3C0319B3290C
:100340002B08DD21A3000310A30DA30DA30DA30D06
:100350000430A9000310A30DA40DA50DA60DA70D33
:10036000A90BAB299B290800061CB42906115030A3
:10037000A100000000000000A10BBA29061CB4294E
:100380000830A900AB01402200000310061C031432
:10039000AB0CA90BC3292B08D221AB00FF212B08E2
:1003A00006150800A30061302302031CDB29230883
:1003B0007A3C0318A312230808002D14A300303040
:1003C000A302031C2D102308163C031C2D102D1C0A
:1003D000A30123081F39A3002308093C0318F229AD
:1003E0000730A30223080F390800303EA300393C30
:1003F0000318FC290730A3072308FF210800A300E6
:10040000861540220830A90000000000A30C031844
:100410008611031C86154022A90B062A861140224C
:100420000000000000000000000000000800270895
:10043000AC002C0E0F394722FF212C080F39472220
:10044000FF212608AC002C0E0F394722FF212C0873
:100450000F394722FF212508AC002C0E0F39472207
:10046000FF212C080F394722FF212408AC002C0E55
:100470000F394722FF212C080F394722FF2108009E
:10048000EA30A10000000000A10B422A0800303E23
:10049000A300393C03184E2A0730A307230808009D
:1004A00083161C158B1355309D00AA309D009C149B
:1004B0008B1783128C1F5A2A8C1383169C1083125D
:0C04C00008000D30FF210A30FF21080069
:10060000AE0003308A001030013E2E02AF001023EE
:10061000FF3903190F2BFF212F08013E062B08007D
:1006200082070D340A34473434344A344E34543457
:1006300020344634723465347134753465346E3424
:1006400063347934203463346F346E3474347234E8
:100650006F346C346C3465347234203466346F34E7
:1006600072342034413444343934383435343134FC
:1006700020344434443453342034203400340D3492
:100680000A345B3452345D3465346134643420346C
:100690004534453420346434613474346134203456
:1006A0002F3420345B3447345D346F342034743459
:1006B0006F34203444344434533420342F342034C1
:1006C00041346E34793420346F3474346834653492
:1006D000723420346B3465347934203474346F349C
:1006E00020346334683461346E34673465342034C4
:1006F000453445342E342034203400340D340A344B
:1007000045346E3474346534723420344134643486
:1007100064347234653473347334203420343034A8
:10072000203474346F342034463420342034003480
:100730000D340A3445346E347434653472342034E4
:10074000343420346234793474346534733420346E
:100750006F3466342034483465347834203444347B
:1007600061347434613420342B3420345B3463348A
:1007700072345D342034203400340D340A345B3458
:1007800057345D34723469347434653420342F3412
:1007900020345B3441345D3462346F3472347434E9
:1007A0002034203400340D340A3444344434533477
:1007B00020344F34703465347234613474346934A5
:1007C0006E3467340D340A3400340D340A34413445
:0C07D0004434443452342E3420340034BD
:02400E00623F0F
:104200001A00AA00AA00AA0015002D002D002D00FA
:104210001200DE00A900D3001500E1005E001500C9
:10422000180009009D00720014008F00EF008C0040
:104230001400F000D10068001900ED004100D0002A
:104240001400B30068003100170010002400E600DD
:104250001800BB00FB000D001400D00021004D0031
:1042600015001100E800D2001A0006008F0085003A
:1042700018003A002500250014008F00EF008C0084
:00000001FF
